:020000020000FC
:100000000C949C030C94B4050C9498050C949C03DC
:100010000C949C030C949C030C9403030C949C037D
:100020000C949C030C949C030C949C030C949C03D4
:100030000C949C030C949C030C949C030C949C03C4
:100040000C94AA050C949C030C949C030C949C03A4
:100050000C949C030C949C030C949C030C949C03A4
:100060000C949C030C949C03475053444F205954C8
:100070002076312E31200400436F756E74730400B6
:1000800077616974203135206D696E202020202031
:1000900004005075736820627574746F6E202020A0
:1000A00020200400746F2070617373200400506876
:1000B000312C2020202031732C200400436F756EDA
:1000C00074696E672E2E2031732073616D706C65BC
:1000D00004005068322C2020203130732C20040082
:1000E0005068332C2020203630732C2004005068B8
:1000F000342C2020323030732C2004003A290400A4
:1001000020202020202020202020202020202020EF
:1001100004004E6F2070756C736520202020202015
:100120002020040053656C662072756E6E696E67E0
:100130002E2E2E20040053657420746F20446566B3
:1001400061756C7420200400436F6E6669672046F9
:100150006F756E642020202004004E6F20636F6E48
:100160006669672020202020202004005365742029
:1001700050574D20746F20353025202004003078F2
:1001800004005068352C2020393030732C200400B6
:100190005068362C2031303030732C2004005361ED
:1001A00074206C6F636B6564203D2004040057610C
:1001B000726D696E67202620536174202020040030
:1001C00057616974696E672E2E2E20202020202012
:1001D000040031302C3030302C3030302E30303084
:1001E000487A040052756E2C2031303030732C2048
:1001F00004003031323334353637383941424344E4
:10020000454603E008B91ED003E008B91BD003E05F
:1002100008B918D002E008B915D002E008B912D028
:1002200094D008E008B90ED000E008B90BD00CE07B
:1002300008B908D000E008B905D006E008B902D036
:100240000BD008954598449A80D044980895459AD3
:10025000449A75D04498089500E008B9F3DF01E0AE
:1002600008B9F0DF089508E008B9ECDF00E008B94C
:10027000E9DF08950CE008B9E5DF00E008B9E2DF46
:10028000089508950CE008B9DDDF0EE008B9DADF63
:10029000089508E008B9D6DF0CE008B9D3DF089567
:1002A00000E205D00895F1E0E0E039D00895102F84
:1002B00002950F701F7008B9CADF18B9C8DF08951A
:1002C0000093210113E018B9C2DF0091210110EF62
:1002D0000123029508B9BBDF13E018B9B8DF00911C
:1002E00021011FE0012308B9B2DF08950093210125
:1002F00013E018B9ACDF0091210110EF0123029542
:1003000008B9A5DF08950093210113E018B99FDF14
:10031000009121011FE0012308B999DF0895C895D4
:10032000002D043059F0002D102D02950F701F7014
:1003300008B98DDF18B98BDF3196F1CF089526EA21
:100340002A95F1F700000000089531E229EC2A9582
:10035000F1F73A95D9F700000000089584DFF0E046
:10036000EEEADDDF08957FDFF0E0E2EDD8DF08950B
:100370007ADFF0E0E0EED3DF089575DFF0E0EEEE37
:10038000CEDF089570DFF1E0E2E8C9DF08956BDFAA
:10039000F1E0E0E9C4DF08956DDFF1E0E2EDBFDFF9
:1003A000089561DFF1E0E4EEBADF08956BDFF0E07D
:1003B000ECEFB5DF08950F9302950F70F1E0E2EFD7
:1003C000E00F08F4F395C895002D71DF0F910F70C1
:1003D000F1E0E2EFE00F08F4F395C895002D67DF38
:1003E00008958827579F402C512C469F202C312C54
:1003F000569F300C411C581E479F300C411C581E04
:100400000895400F511F621F731F0895112722275F
:100410003327BB27AA279927881BC1E277956795C1
:1004200057954795CA9551F020F4800F911FA21F50
:10043000B31FB795A79597958795F0CF0895002797
:100440001127222733274427552766277727882710
:100450009927AA27BB27CC27DD27EE27FF2708955A
:10046000A89572E486ED9BEE9A95F1F78A95D9F7F7
:100470007A95C1F773E07A95F1F700000895DD27CA
:10048000CC2701E000930201EBDF2ED1A89500916B
:100490000201003021F02196CA17DB07A8F30027DC
:1004A000009302010895DD27CC275527662777277B
:1004B00088279927C8E20ED0000F111F221F331F73
:1004C000441F551F661F771F881F991FAA1FCA95B3
:1004D00091F708955F935F70553010F05D5FD52FF1
:1004E000D52F5F91507F503508F0505D5D0F6F93B1
:1004F0006F70653010F06D5FD62FD62F6F91607FD3
:10050000603508F0605D6D0F7F937F70753010F07F
:100510007D5FD72FD72F7F91707F703508F0705D8A
:100520007D0F8F938F70853010F08D5FD82FD82F6F
:100530008F91807F803508F0805D8D0F9F939F7035
:10054000953010F09D5FD92FD92F9F91907F9035D6
:1005500008F0905D9D0F0895AF93AF70A53010F037
:10056000AD5FDA2FDA2FAF91A07FA03508F0A05D44
:10057000AD0F0895F999FECF112711BD12BDF1E01D
:10058000EBE2019100BD04E00FBBFA9AF99AF999E8
:10059000FECF139511BD1230A1F711270895F999D7
:1005A000FECF1127009134010F3F19F402E00093B0
:1005B0003401112712BD01BDF1E0E9E0019100BD58
:1005C00004E00FBBFA9AF99AF999FECF139511BD81
:1005D0001130A1F70091340103950093340108957F
:1005E000F999FECFAA27BB27A1BDB2BDF1E0EBE28E
:1005F000F89AF899FECF00B501931196A1BDB2BD4E
:10060000A230B1F70895A895F89401E000932D0168
:1006100000910301063009F012C025DEF1E0E4E2AA
:100620007EDE28DEF1E0E2ED7ADEDADF00912B01FA
:100630000093890000912C010093880009C00CDE12
:1006400012DEF1E0E2E16BDE15DEF1E0E4E267DE0E
:1006500001E005BB00E005BDF2DE002706BD00930A
:1006600000010093010193C3BB27AA27F999FECF8C
:10067000B2BDA1BD0FEF00BDFA9AF99AA395B1F7EB
:10068000089510E000E41093C5000093C40008E151
:100690000093C10006E00093C20008951091C000CD
:1006A00017FFFCCF0091C60008951091C00015FF00
:1006B000FCCF0093C6000895A895F0DF0734E1F75A
:1006C000EDDF0734C9F7EADF0134B1F72227E6DFAF
:1006D0000C32E9F723952730D1F7E0DF009336019C
:1006E000DDDF0093370108950091C00007FF0895F2
:1006F00000913801013009F008952196DDDFBADD5F
:10070000F1E0EEE90CDE00913601D1DD0091370118
:10071000CEDDC6DD08950091C00007FF0895CCDF4F
:10072000B8DD03E5C4DD0DE3C2DD00913601BFDDB8
:1007300000913701BCDD08950FEF0DBF08E00EBF3B
:100740000FEF04B907B900270AB908B90FEF0BB9C1
:1007500002E00DBB0BE00093690002E0009334015E
:100760000027009338014DDD77DD7DDDF0E0E8E620
:10077000D6DDBB27A5E083DE84DF0FEF0093870083
:100780000FEF0093860002E80093800009E10093D8
:1007900081004B9909C060DD66DDF1E0E6E3BFDD75
:1007A00063DFBB27A5E06BDE1BDF10912C012091DE
:1007B0002B010FEF10172007F1F000912B01009390
:1007C000890000912C010093880046DD4CDDF1E0AA
:1007D000E8E4A5DD4FDDF1E0EEE7A1DD00912B01BE
:1007E000EADD00912C01E7DDBB27A5E048DE06E04D
:1007F0000093030115C00FE7009389000FEF0093EA
:1008000088002ADD30DDF1E0EAE589DD33DDF1E065
:10081000ECE685DDBB27A5E032DE01E000930301B5
:1008200001E000936E0000E005BD002706BD0093C7
:1008300000010093010180D202DEA89508E1009337
:10084000600006E40093600000910301063049F067
:1008500001E000932E01002700932F017FDD5BDF75
:1008600096C295DD58DF98DD08EE00932E0103E077
:1008700000932F018CC272DD4EDF00910901003818
:1008800061F0EAF030918900209188002D533A40C0
:1008900030938900209388007AC288DDB0E0A5E01B
:1008A000EEDDE8DC00DD5FDD36DF02E00093030112
:1008B0000AE000932E01002700932F0168C2B09137
:1008C0008900A09188000DE31AE0A00FB11FB0933A
:1008D0008900A09388005BC246DD1DDF0AE000931B
:1008E0002E01002700932F0100910901003089F0AB
:1008F000009109010233F8F0B0918900A0918800BD
:1009000006E011E0A00FB11FB0938900A09388000A
:100910003EC24CDDB0E0A5E0B2DDACDCC4DC28DDDD
:10092000FADE03E0009303010CE300932E0100279D
:1009300000932F012CC2309189002091880026500D
:100940003140309389002093880021C211DDE3DE1D
:100950000CE300932E01002700932F010091090161
:10096000003079F00F37F8F0B0918900A09188003D
:100970000BE210E0A00FB11FB0938900A093880094
:1009800006C214DDB0E0A5E07ADDF7DCC4DE72DC7F
:100990008ADC04E00093030108EC00932E01002799
:1009A00000932F01F4C130918900209188002B52CF
:1009B00030403093890020938800E9C1DEDCABDE53
:1009C00008EC00932E01002700932F0100910901EC
:1009D000003079F00F37F8F0B0918900A0918800CD
:1009E0000CE010E0A00FB11FB0938900A093880025
:1009F000CEC1DCDCB0E0A5E042DDC4DC8CDE3ADC5C
:100A000052DC05E00093030104E800932E0103E0AB
:100A100000932F01BCC130918900209188002C5097
:100A200030403093890020938800B1C1ABDC73DE85
:100A3000B6DD04E800932E0103E000932F0100913E
:100A40000901003081F00F3768F0B0918900A09162
:100A5000880003E010E0A00FB11FB0938900A093BD
:100A6000880095C112C0A2DCB0E0A5E008DD8FDCF3
:100A700052DE00DC18DC06E00093030108EE009370
:100A80002E0103E000932F0182C1B0918900A09153
:100A90008800A350B040B0938900A093880077C12C
:100AA000009109017CDD9CDD10912C0120912B012E
:100AB0000FEF1017200711F074DC01C068DC2BDE8B
:100AC00008EE00932E0103E000932F01009109012D
:100AD000003081F00F3768F0B0918900A091880054
:100AE00002E010E0A00FB11FB0938900A09388002E
:100AF0004EC113C0309189002091880030932B01A2
:100B000020932C0137DD06E00093030108EE0093EB
:100B10002E0103E000932F013AC1B0918900A0910A
:100B20008800A250B040B0938900A09388002FC1E4
:100B30000F930FB70F9300910201013039F4002792
:100B4000009302010F910FBF0F9118950F910FBFE6
:100B50000F9118950FEFA017B00711F01196189587
:100B60002196AA27BB271895009101011091000139
:100B700020912F0130912E011317020769F0A895DB
:100B800001E005BDF0910101E09100013196F09383
:100B90000101E0930001189500E005BD00270093D6
:100BA000010100930001A895F8945B2F4A2F71E092
:100BB00060E017DC2F923F924F925F92DF93CF93CA
:100BC0003EDCCF91DF914C2F5D2F31E022DC3F9155
:100BD0002F911F910F919927400F511F621F731F73
:100BE000891F06B51127222733279927400F511F48
:100BF000621F731F891FA89B0CC001E005BB002763
:100C000011E0222733279927400F511F621F731FBE
:100C1000891F4093090150930A0160930B0170935F
:100C20000C0180930D0140910D0130910C01209138
:100C30000B0110910A010091090135DC509322014A
:100C400060932301709324018093250190932601E2
:100C5000A09335010FDB27DB0DDB0091030106308C
:100C600081F0009126012CDB0091250129DB009108
:100C7000240126DB0091230123DB0091220120DBEC
:100C800028C000913501003011F40ADB03C0009147
:100C9000350139DB0091260129DB0CE208DB0091EC
:100CA000260131DB009125010BDB0CE200DB00911A
:100CB000240106DB0091230119DB0EE2F8DA009132
:100CC000230121DB00912201FBDA08E4F0DA0AE7D4
:100CD000EEDAB5DB06BD009300010093010100913F
:100CE0000301013029F40FEF0DBF08E00EBFC3CDA3
:100CF000023029F40FEF0DBF08E00EBFEDCD033039
:100D000029F40FEF0DBF08E00EBF20CE043029F408
:100D10000FEF0DBF08E00EBF51CE053029F40FEFE5
:100D20000DBF08E00EBF82CE063029F40FEF0DBFD5
:100D300008E00EBFB5CE18958FDA95DAF1E0EEEA4D
:100D4000EEDA98DAF0E0E0E8EADAB0E0A5E097DB86
:100D500083DA89DAF0E0E2E9E2DA8CDAF0E0E4EA78
:100D6000DEDAB0E0A5E08BDB77DA7DDAF1E0E0EC0B
:100D7000D6DAB3E0A4E801E000933801A8957894AE
:100D80007EDB002700933801F89466DA089568DB6B
:100D900067DB55DB01E00CBB01E00DBBA895789447
:100DA0000000000000000000000000000000000043
:100DB0000000000000000000000000000000000033
:100DC0000000000000000000000000000000000023
:100DD0000000000000000000000000000000000013
:041D600000001EC899
:00000001FF
